:0200000480007A
:1000000017110000130101001309000093080000FC
:10001000B308190323201101130A000093091000EB
:10002000B3093A0323223101130B0000930AF0FFB6
:10003000B30A5B0323245101130C0000B70B0080AB
:10004000938BFBFFB30B7C0323267101130D000080
:10005000B70C0080B30C9D032328910117110000F9
:10006000130181FB130E1000930D0000B30DBE03AE
:100070002320B101130F1000930E1000B30EDF0305
:100080002322D10193011000930FF0FFB38FF103EE
:100090002324F10113041000370200801302F2FF41
:1000A000330244022326410093051000B704008068
:1000B000B38495022328910017110000130101F762
:1000C0009306F0FF130600003386C6022320C1000A
:1000D0009307F0FF130710003387E7022322E100A4
:1000E0009308F0FF1308F0FF33880803232401016D
:1000F0009309F0FF370900801309F9FF33892903B9
:1001000023262101930AF0FF370A0080338A4A032D
:100110002328410117110000130181F2B70B008061
:10012000938BFBFF130B0000338B6B0323206101C8
:10013000B70C0080938CFCFF130C1000338C8C03E5
:1001400023228101B70D0080938DFDFF130DF0FF79
:10015000338DAD032324A101B70E0080938EFEFFE3
:10016000370E0080130EFEFF338ECE032326C1010F
:10017000B70F0080938FFFFF370F0080338FEF039F
:100180002328E101171100001301C1EC37020080A0
:1001900093010000B301320223203100B704008034
:1001A0001304100033848402232281003706008068
:1001B0009305F0FFB305B6022324B1003707008092
:1001C000B70600809386F6FFB306D7022326D10038
:1001D00037080080B7070080B307F8022328F10032
:1001E00017150000130505E297150000938585EEAD
:1001F000370610F01306C6F26306B5028326C50063
:100200002320D600832685002320D60083264500A0
:100210002320D600832605002320D60013050501E0
:100220006FF09FFD370510F0130505F22320050040
:0402300000000000CA
:10100000FFFFFFFFFFFFFFFFFFFFFFFFFFFFFFFFF0
:10101000FFFFFFFFFFFFFFFFFFFFFFFFFFFFFFFFE0
:10102000FFFFFFFFFFFFFFFFFFFFFFFFFFFFFFFFD0
:10103000FFFFFFFFFFFFFFFFFFFFFFFFFFFFFFFFC0
:10104000FFFFFFFFFFFFFFFFFFFFFFFFFFFFFFFFB0
:10105000FFFFFFFFFFFFFFFFFFFFFFFFFFFFFFFFA0
:10106000FFFFFFFFFFFFFFFFFFFFFFFFFFFFFFFF90
:10107000FFFFFFFFFFFFFFFFFFFFFFFFFFFFFFFF80
:10108000FFFFFFFFFFFFFFFFFFFFFFFFFFFFFFFF70
:10109000FFFFFFFFFFFFFFFFFFFFFFFFFFFFFFFF60
:1010A000FFFFFFFFFFFFFFFFFFFFFFFFFFFFFFFF50
:1010B000FFFFFFFFFFFFFFFFFFFFFFFFFFFFFFFF40
:1010C000FFFFFFFFFFFFFFFF000000000000000028
:040000058000000077
:00000001FF
